:06000000028081028188EC
:03000B00028188E7
:03001300028188DF
:03001B00028188D7
:03002300028188CF
:03002B00028188C7
:0E0032003830353164756D7065722076312E70
:1000400030206279204E4636580D0A004552524FF4
:10005000523A20436F756C64206E6F742072656134
:100060006420524F4D2073697A65206B6E6F622158
:100070000D0A003A303030303030303146460D0A0B
:100080000075A8007590FF758160C2907587007536
:100090009850758921758DFD758BFDD28E908032BB
:1000A00031AFC292318E309318D292318E3093118B
:1000B000318E30930C318E309307318E3093028025
:1000C000E1D292209405753080802020950575300E
:1000D00040801820960575302080102097057530D7
:1000E00010800890804C31AF02818875343A7535A4
:1000F00031753630755E0D755F0A756000900000D1
:10010000E583B53002802EB2917531107837E583E2
:100110003140E5823140E43140E4933140E582549E
:100120000FC3940F6003A380F0E531F42401314044
:100130003178A380CB90807331AFC292D29180FE90
:10014000F532F5332531F531E532C4540F2430F55D
:1001500032C3943A4006E5322407F532E533540FB2
:100160002430F533C3943A4006E5332407F533E5EC
:1001700032F608E533F608227834E6600AC299F5CB
:10018000993099FD0880F322D292C29180FEC28CF0
:10019000758C4C758A00C28DD28C308DFDC28C75E9
:1001A0008C4C758A00C28DD28C308DFDC28C22E4BD
:0E01B00093600AC299F5993099FDA380F2225E
:00000001FF
